:1000000092C0AAC0A9C0A8C0A7C0A7C0A5C0A4C0CC
:10001000A3C0A2C0A1C0A0C09FC09EC09DC09CC0E4
:100020009BC09AC099C000000000010101020203B8
:100030000405050607090A0B0C0E0F1112141517FB
:10004000191B1D1F212325282A2C2F313436393B1B
:100050003E414346494C4F5255585A5D6164676A68
:100060006D707376797C7F8386898C8F9295989B4F
:100070009EA2A5A7AAADB0B3B6B9BCBEC1C4C6C93D
:10008000CBCED0D3D5D7DADCDEE0E2E4E6E8EAEBAB
:10009000EDEEF0F1F3F4F5F6F8F9FAFAFBFCFDFDFC
:1000A000FEFEFEFFFFFFFFFFFFFFFEFEFEFDFDFC6D
:1000B000FBFAFAF9F8F6F5F4F3F1F0EEEDEBEAE815
:1000C000E6E4E2E0DEDCDAD7D5D3D0CECBC9C6C4D5
:1000D000C1BEBCB9B6B3B0ADAAA7A5A29E9B989568
:1000E000928F8C898683807C797673706D6A676461
:1000F000615D5A5855524F4C494643413E3B393653
:1001000034312F2C2A282523211F1D1B19171514C4
:1001100012110F0E0C0B0A09070605050403020253
:1001200001010100000011241FBECFEDCDBF10E082
:10013000A0E6B0E0EEE2F5E003C0C89531960D927E
:10014000A238B107D1F710E0A2E8B0E001C01D92DB
:10015000A03CB107E1F768C153CF1F920F920FB6D1
:100160000F9211242F933F934F935F936F937F933D
:100170008F939F93AF93BF93CF93DF93EF93FF93AF
:1001800060918200615060938200662329F480911F
:1001900083008F5F8093830010928B0010928A00FF
:1001A00020916200209389002D3008F04CC0A22FCE
:1001B000BB27AA0FBB1FDB2FCA2FC457DF4F4881B5
:1001C00059814F3F510509F008F43DC0FB2FEA2F3C
:1001D000EA55FF4FA959BF4F808191812D913C91E4
:1001E000820F931F9183808380589F4F9093880044
:1001F00080938700E92FFF27EA5DFF4FC895202DE8
:10020000332730938B0020938A00841B950B8050FA
:100210009048E92FFF27EA5DFF4FC895802D280FF2
:10022000311D30938B0020938A006623B1F4952F03
:10023000842FB4E096958795BA95E1F7481B590B42
:10024000598348830AC080918A0090918B00805026
:100250009F4F90938B0080938A00209161002093A0
:1002600089002D3008F053C0A22FBB27AA0FBB1F57
:10027000DB2FCA2FC457DF4F688179816F3F71052B
:1002800009F008F444C0FB2FEA2FEA55FF4FA959A3
:10029000BF4F808191812D913C91820F931F91835B
:1002A000808380589F4F9093880080938700E92F28
:1002B000FF27EA5DFF4FC895402D20918A003091BD
:1002C0008B00240F311D30938B0020938A00861BF6
:1002D000970B80509048E92FFF27EA5DFF4FC895A4
:1002E000802D280F311D30938B0020938A00809140
:1002F00082008823B1F4972F862FE4E096958795A6
:10030000EA95E1F7681B790B798368830AC08091CD
:100310008A0090918B0080509F4F90938B00809328
:100320008A0020916000209389002D3008F053C08E
:10033000A22FBB27AA0FBB1FDB2FCA2FC457DF4F2B
:10034000688179816F3F710509F008F444C0FB2F83
:10035000EA2FEA55FF4FA959BF4F808191812D9116
:100360003C91820F931F9183808380589F4F90937D
:10037000880080938700E92FFF27EA5DFF4FC8952B
:10038000402D20918A0030918B00240F311D309335
:100390008B0020938A00861B970B80509048E92F92
:1003A000FF27EA5DFF4FC895802D280F311D309340
:1003B0008B0020938A00809182008823B1F4972FCC
:1003C000862F34E0969587953A95E1F7681B790B6F
:1003D000798368830AC080918A0090918B00805055
:1003E0009F4F90938B0080938A0080918A00909118
:1003F0008B0023E0969587952A95E1F788BD88B50F
:100400008ABDFF91EF91DF91CF91BF91AF919F9105
:100410008F917F916F915F914F913F912F910F90AD
:100420000FBE0F901F901895CFEDD0E0DEBFCDBF6F
:1004300087EF88BB88E187BB8FE782BB11BA81EB6E
:100440008FBD81E08EBD80E889BF78948091830064
:100450008823E1F38150809383004091650050919F
:100460006600509364004093630086B3282F3327BF
:100470002770307086B39927807E90709595879508
:1004800095958795282B392B80B399278F77907076
:10049000F6E0880F991FFA95E1F7282B392B309356
:1004A000660020936500932F822F8095909584237A
:1004B0009523909385008093840010928600C1E07C
:1004C000D0E0682F792FA0E0B0E820E050916000E4
:1004D00040916100309162008C2F9D2F022E02C04E
:1004E000880F991F0A94E2F786239723892B89F0B6
:1004F000251739F0241729F0231719F0542F432F0B
:10050000322FE22FFF27EE0FFF1FE457FF4FB1837B
:10051000A083822F8F5F282F8D30F0F230936200FE
:0E0520004093610050936000809386008FCF5F
:10052E00FFFFFFFF00FF008A080C099509270AC28A
:10053E000A660B130CCB0C8E0D5C0E370F1E1014AF
:02054E0011009A
:00000001FF
